:0200000480007A
:100000009705000093850502130540006B10B500AD
:10001000EF000001EF00404D130500006B000500EC
:10002000130540006B000500F32610029396F600BE
:10003000732600029315A6001316260037F1FF6FF2
:100040003301B1403301D1403301C100F326100226
:1000500063860600130500006B0005006780000042
:100060006B10B500678000006B0005006780000022
:100070006B40B500678000006B20050067800000C2
:100080006B3000006780000073251002678000005D
:100090007325000267800000130141FF2320110037
:1000A0002322B1008345050063880500EF00C001ED
:1000B000130515006FF01FFF832001008325410009
:1000C0001301C10067800000B702010023A0B20045
:1000D00067800000130101FE232E1100232C8100F4
:1000E000130401022326A4FEB70700810327C4FEE0
:1000F000131727009387870EB307F70083A707001E
:1001000013850700EFF05FF9130000008320C101A1
:10011000032481011301010267800000130101FE25
:10012000232E1100232C8100130401022326A4FE98
:100130002324B4FE0325C4FEEFF01FF6032584FE3E
:10014000EFF05FF9B707008113850704EFF0DFF4E4
:10015000130000008320C101032481011301010267
:1001600067800000130101FE232E1100232C810063
:1001700013040102B707008113854708EFF0DFF190
:1001800013054000EFF05FEEEFF09FF02326A4FE92
:100190000327C4FEB70700818326C4FE939626007A
:1001A0009387871AB387F60023A0E7001305100092
:1001B000EFF09FEBB707008183A7871A138507002D
:1001C000EFF05FF1B707008113850709EFF0DFEC6F
:1001D000B70700819387871A83A747001385070015
:1001E000EFF05FEFB707008113850709EFF0DFEA53
:1001F000B70700819387871A83A7870013850700B5
:10020000EFF05FEDB707008113850709EFF0DFE836
:10021000B70700819387871A83A7C7001385070054
:10022000EFF05FEBB707008113850709EFF0DFE61A
:10023000130000008320C101032481011301010286
:1002400067800000130101FE232E1100232C810082
:1002500013040102EFF0DFE32326A4FE8327C4FE8C
:1002600093B72700A305F4FE8347B4FE1385070068
:10027000EFF09FE08347B4FE638407068327C4FE44
:1002800093B717002305F4FE8347A4FE13850700E8
:10029000EFF09FDE8347A4FE63820702B707008169
:1002A0000327C4FE131727009387871AB307F700A5
:1002B0001307A00023A0E7006F000002B70700812A
:1002C0000327C4FE131727009387871AB307F70085
:1002D0001307B00023A0E700EFF09FDA6F0040069D
:1002E0008327C4FE93B73700A304F4FE834794FE2C
:1002F00013850700EFF05FD8834794FE63820702FF
:10030000B70700810327C4FE131727009387871AB6
:10031000B307F7001307C00023A0E7006F00000237
:10032000B70700810327C4FE131727009387871A96
:10033000B307F7001307D00023A0E700EFF05FD466
:10034000EFF01FD4B707008183A7871A1385070032
:10035000EFF05FD8B707008113850709EFF0DFD30F
:10036000B70700819387871A83A747001385070083
:10037000EFF05FD6B707008113850709EFF0DFD1F3
:10038000B70700819387871A83A787001385070023
:10039000EFF05FD4B707008113850709EFF0DFCFD7
:1003A000B70700819387871A83A7C70013850700C3
:1003B000EFF05FD2B707008113850709EFF0DFCDBB
:1003C000130000008320C1010324810113010102F5
:1003D00067800000130101FE232E1100232C8100F1
:1003E00013040102EFF05FCA2326A4FEB7070081C1
:1003F0000327C4FE131727009387871BB307F70053
:100400000327C4FE23A0E7008327C4FE63860700FA
:1004100013050000EFF05FC5130000008320C10149
:10042000032481011301010267800000130101FE12
:10043000232E1100232C810013040102B707008032
:100440009387473D2326F4FE8325C4FE1305400011
:10045000EFF01FC1EFF01FF8B707008183A7871BDC
:1004600013850700EFF01FC7B70700811385070941
:10047000EFF09FC2B70700819387871B83A74700D0
:1004800013850700EFF01FC5B70700811385070923
:10049000EFF09FC0B70700819387871B83A7870072
:1004A00013850700EFF01FC3B70700811385070905
:1004B000EFF09FBEB70700819387871B83A7C70014
:1004C00013850700EFF01FC1B707008113850709E7
:1004D000EFF09FBC130000008320C10103248101C1
:1004E0001301010267800000130101FF23261100A0
:1004F000232481001304010113051000EFF0DFB67F
:10050000EFF05FC6B70700811385470DEFF0DFB846
:1005100013054000EFF05FB5EFF0DFD213051000D8
:10052000EFF09FB493070000138507008320C100FC
:0C0530000324810013010101678000001A
:02000004810079
:10000000300000003100000032000000330000002A
:10001000340000003500000036000000370000000A
:10002000380000003900000061000000620000009C
:10003000630000006400000065000000660000002E
:100040000A00000030000000310000003200000013
:1000500033000000340000003500000036000000CE
:100060003700000038000000390000006100000087
:1000700062000000630000006400000065000000F2
:1000800066000000746573745F746D630A0000009D
:100090000A000000300000003100000032000000C3
:1000A000330000003400000035000000360000007E
:1000B0003700000038000000390000006100000037
:1000C00062000000630000006400000065000000A2
:1000D00066000000746573745F64697665726765B5
:0500E0006E63650A00DB
:1000E8000000008104000081080000810C000081EC
:1000F8001000008114000081180000811C0000819C
:100108002000008124000081280000812C0000814B
:100118003000008134000081380000813C000081FB
:1001280044000081480000814C000081500000819B
:1001380054000081580000815C000081600000814B
:1001480064000081680000816C00008170000081FB
:1001580074000081780000817C00008180000081AB
:1001680094000081980000819C000081A00000811B
:10017800A4000081A8000081AC000081B0000081CB
:10018800B4000081B8000081BC000081C00000817B
:10019800C4000081C8000081CC000081D00000812B
:040000058000000077
:00000001FF
